:020000040000FA
:1000000097223F2B820750344934433453344D34C4
:1000100054342034763431342E34313400341030BA
:10002000BF00C101C0012030BB008620440803107E
:10003000C1070318C00ABF0B1528A7014008A60076
:100040004108A5009E207D30AF002030AE00AD01FC
:10005000AC0175218830AF00AA30AE00AD01AC0113
:10006000E0211A212708C6002608C7002508C80075
:10007000A71F3F28A709A609A5092D30BB00260800
:10008000A7002508A6000330B5003E306A224608C6
:10009000A7004708A6004808A5009E207C30AF00B6
:1000A0003830AE005130AD00EC30AC0075218430FA
:1000B000AF00AE01AD01AC01E0211A21C601A71FBE
:1000C0006528A709A609A50946142508A600033036
:1000D000B50038306A222D304618B6000930E622C5
:1000E00036089F2237089F2238089F220A30E622CE
:1000F0003B089F223C089F223D089F222E309F22D2
:100100003E089F2243309F22AD22F02A2030C300B8
:100110003630C200C501C40103110000061AC50A29
:100120000319C40AC30B8D28C20B8E280310C50DFA
:10013000C40DC50DC40DC50DC40D08009630A80032
:10014000A901A71FAC28A509A609A709A50A031993
:10015000A60A0319A70AA917B3012708031DC12876
:100160002608A7002508A600A501B3152708031D2A
:10017000C1282608A700A601B311331627080319C2
:10018000D2283308A802031D031CD3290310A71B80
:10019000CF28A50DA60DA70DA80BC728D329A91FE9
:1001A000A7130034A701A601A501A401A8010034EA
:1001B000B3012708031DF8282608A7002508A60074
:1001C0002408A500A401B3152708031DF828260854
:1001D000A7002508A600A501B31133162708031DA3
:1001E000F8282608A700A601B31527080319D22866
:1001F0003308A802031D031CD3290310A71B0729DA
:10020000A40DA50DA60DA70DA80BFE28D3292A1B0A
:10021000251CCF28A41FCF28A50A0319A60A031955
:10022000A70A031DCF28A70CA60CA50CA80A031922
:10023000C829CF282808031900342708A900A717C0
:100240009630A802A81F6929A809A80A0830280220
:10025000031C4529A800A50D2608A5002708A6000F
:10026000A70108302802031C4529A800A50D26086F
:10027000A500A60108302802031C4529A800A50DE9
:10028000A5012808031D03104E29280803194E292B
:100290000310A70CA60CA50CA80B48292A1B251C8B
:1002A0005A29031C5A29A50A0319A60A0319A70AE1
:1002B000A71B6929A91F0034A709A609A509A50A32
:1002C0000319A60A0319A70A0034A701A601A5016C
:1002D00000342A14AA1FFF34A701A91FFF30A7006A
:1002E000A600A500A90DA70CFF342808031D2F08A0
:1002F0000319D22827082E06A9002F08A8077E3048
:10030000031C8629A8020318C8298929A802031CEE
:10031000D3292708A4002608A3002508A200A417B3
:10032000AE170310A701A601A5011830B300221CC7
:10033000A3292C08A5072D0803182D0FA6072E08A2
:1003400003182E0FA707A70CA60CA50CA40CA30C32
:10035000A20C0310B30B9729A71BB329A40DA50D5D
:10036000A60DA70DA8032A1B251CC529A41FC52956
:10037000A50A0319A60A0319A70A031DC529A70C74
:10038000A60CA50CA80A0319C829A91FA713003495
:10039000AA14AA1FFF34FF30A800A700A600A500DA
:1003A000A90DA70CFF342A15AA1FFF340130A8009D
:1003B000A701A601A501A90DA70CFF348030AE0648
:1003C00027082E06B300A401AB0128082F02031C46
:1003D000012A2F08A2002808AF002208A8002E0832
:1003E000A2002708AE002208A7002D08A2002608B8
:1003F000AD002208A6002C08A2002508AC002208A7
:10040000A5002F08031900342708A900A717AE1765
:100410002F082802AF000319342A08302F02031CCA
:100420002A2AAF002C08AB002D08AC002E08AD0026
:10043000AE0108302F02031C2A2AAF002C08AB00A3
:100440002D08AC00AD0108302F02031C2A2A290810
:10045000A70000342F080319342A0310AE0CAD0C8A
:10046000AC0CAB0CAF0B2D2AB31F412AAB09AC0966
:10047000AD09AE09AB0A0319AC0A0319AD0A031999
:10048000AE0A2B08A4072C0803182C0FA5072D086B
:1004900003182D0FA6072E0803182E0FA707B31B4E
:1004A0005A2A031C0729A70CA60CA50CA40CA80FFC
:1004B0000729C8290318D828A409A509A609A70946
:1004C000A40A0319A50A0319A60A0319A70A80306A
:1004D000A906AC288400AE010A30AD0077222208BC
:1004E0008000303080078403B50B6B2A0800A3011D
:1004F000A2011030B400270DA20DA30D2D08A202F9
:100500002E08031C2E0FA30203188D2A2D08A20704
:100510002E0803182E0FA3070310A60DA70DB40B6A
:100520007B2A0034CA000000CA0B942A08008316F4
:100530008511831285110830CF22C9000800CC0034
:100540000A30CB0003108511031C8515490892223F
:100550000314CC0CCB0BA32A08000D309F2A0800F3
:100560000A309F2A080020309F2A08004C10051EE0
:1005700000340930CB00490892220310051E0314F1
:10058000CC0C490892220000CB0BBD2A4C08051A5E
:10059000C72A4C140800B6224C1CCB2A08003F394D
:1005A0008900831608148312080808003F3989005F
:1005B00083168B13081555308900AA3089008814DA
:1005C00008118B178818E22A83120800CF22C60070
:1005D0004608CF220038031908009F22C60AE82ADD
:1005E00005190F28B6224C1CC6001B3A0319F92A1C
:1005F000F02ACB22C6001B3A0319F92A4608443ACE
:100600000319242B46084F3A0319172B4608563A6C
:1006100003193F2B4608503A03191D2B4608553A3B
:100620000319312B46084D3A03190F28F02A1430CC
:10063000C7000930CF22C600262B1430C7009F22E6
:100640000930CF22C600352BC601C701CB22880056
:100650004608D622C7030319F02AC60A461F262BCE
:10066000F02A40309F22C601C7014608CF229F22B0
:10067000C7030319F02AC60A461F352BF02AC60104
:100680004608022000380319482B9F22C60A402B37
:06069000AD22B022F02AA9
:02400E00F23F7F
:1042000000000000000000000000000000000000AE
:1042100050000B002C00210035003000300033002E
:104220002E00300030004E002F00300031003400EE
:10423000320037002E003000300045005F003000B3
:10424000300030002F0030003000300067003000B8
:104250003000300074000000580050004900430056
:10426000200053004D0054002000740065006D00D4
:0642700070003A0000009E
:00000001FF
